:1000000019C033C032C031C030C02FC02EC0DBC1D8
:100010002CC02BC0B9C029C028C027C026C025C00D
:1000200024C023C022C021C020C01FC01EC01DC0CC
:1000300063C31BC011241FBECFEFD4E0DEBFCDBF12
:1000400011E0A0E0B1E0EEEDF8E002C005900D9205
:10005000A030B107D9F711E0A0E0B1E001C01D92D6
:10006000A034B107E1F721D038C400C01F920F922D
:100070000FB60F9211240F900FBE0F901F9018957E
:1000800080FF02C05C9A01C05C9881FF02C0439A65
:1000900001C0439882FF02C0589A01C0589883FF5C
:1000A00002C0599A08955998089587E085B918B8FB
:1000B0008CE08BB914B88FE387B983EF8AB98BB121
:1000C0008F718BB98BB1806E8BB980E0D9DF1092C4
:1000D000800080E593EC909387008093860084E114
:1000E0008093B30092E09093B0009093B10010928F
:1000F000800089E1809381009093700080E280937A
:100100006F008CEC8093BA0085E48093BC00F89477
:100110008091000182FF02C080E006C08091000152
:1001200084608093000181E07894882381F378943F
:1001300021E42093070180910101909102019093A5
:10014000090180930801809103019091040190932B
:100150000B0180930A018091050190910601909313
:100160000D0180930C0110920E014A9905C08091F7
:100170000E01816080930E014B99DBCF80910E01BF
:10018000826080930E01D5CF1F920F920FB60F920F
:100190001124EF92FF920F931F932F933F934F934E
:1001A0005F936F938F939F93AF93BF93809123013E
:1001B00090912401A0912501B0912601805B9C4380
:1001C000AF4FBF4F8093230190932401A09325014B
:1001D000B09326018091230190912401A0912501E3
:1001E000B091260180509842AB46BE4E40F010922E
:1001F0002301109224011092250110922601809172
:100200002701883009F0C8C02091230130912401D2
:1002100040912501509126018091840090918500A4
:10022000A0E0B0E0820F931FA41FB51F109227011A
:1002300020911701309118014091190150911A0134
:1002400082179307A407B50748F07C018D01E21AD5
:10025000F30A040B150BA80197010CC07C018D015A
:10026000E21AF30A040B150BA80197012050384D30
:1002700044495141215432444F40504060F0109263
:100280000201109201018093170190931801A0932D
:100290001901B0931A0120911B0130911C0140916A
:1002A0001D0150911E0182179307A407B50748F05E
:1002B0007C018D01E21AF30A040B150BA8019701CA
:1002C0000CC07C018D01E21AF30A040B150BA80186
:1002D00097012050384D44495141215432444F40F8
:1002E000504060F0109204011092030180931B01B2
:1002F00090931C01A0931D01B0931E0120911F013A
:1003000030912001409121015091220182179307E1
:10031000A407B50748F07C018D01E21AF30A040B2B
:10032000150BA80197010CC07C018D01E21AF30A9C
:10033000040B150BA80197012050384D4449514139
:10034000215432444F40504060F010920601109208
:10035000050180931F0190932001A0932101B09388
:1003600022018091110190911201892B11F4409882
:1003700001C0409A8091130190911401892B11F4CE
:10038000419801C0419A8091150190911601892BE5
:1003900011F4429801C0429A809127018F5F8093A7
:1003A0002701BF91AF919F918F916F915F914F9175
:1003B0003F912F911F910F91FF90EF900F900FBEE3
:1003C0000F901F9018951F920F920FB60F92112445
:1003D000EF92FF920F931F932F933F934F935F934F
:1003E0006F937F938F939F93AF93BF93EF93E3B1FB
:1003F000E77080912801E81709F44CC16E2F70E076
:100400008091280190E08627972780FF67C0E0FD54
:100410001BC020912301309124014091250150916E
:1004200026018091840090918500A0E0B0E0820FC9
:10043000931FA41FB51F8093290190932A01A093B5
:100440002B01B0932C014AC0E0902901F0902A01C1
:1004500000912B0110912C01209123013091240156
:100460004091250150912601809184009091850052
:10047000A0E0B0E0820F931FA41FB51F8E159F054B
:10048000A007B10728F08E199F09A00BB10B08C077
:100490008E199F09A00BB10B8050984DA449B14112
:1004A0009093020180930101209123013091240156
:1004B0004091250150912601809184009091850002
:1004C000A0E0B0E0820F931FA41FB51F8093170117
:1004D00090931801A0931901B0931A0180912801FB
:1004E00090E08627972781FF67C061FD1BC02091A0
:1004F00023013091240140912501509126018091E2
:10050000840090918500A0E0B0E0820F931FA41FAB
:10051000B51F80932D0190932E01A0932F01B093CE
:1005200030014AC0E0902D01F0902E0100912F0182
:100530001091300120912301309124014091250137
:10054000509126018091840090918500A0E0B0E058
:10055000820F931FA41FB51F8E159F05A007B1071B
:1005600028F08E199F09A00BB10B08C08E199F09A6
:10057000A00BB10B8050984DA449B1419093040158
:1005800080930301209123013091240140912501A2
:10059000509126018091840090918500A0E0B0E008
:1005A000820F931FA41FB51F80931B0190931C0102
:1005B000A0931D01B0931E018091280190E0862731
:1005C000972782FF67C062FD1BC0209123013091F5
:1005D0002401409125015091260180918400909141
:1005E0008500A0E0B0E0820F931FA41FB51F809389
:1005F000310190933201A0933301B09334014AC08A
:10060000E0903101F09032010091330110913401FA
:100610002091230130912401409125015091260120
:100620008091840090918500A0E0B0E0820F931F3C
:10063000A41FB51F8E159F05A007B10728F08E19BE
:100640009F09A00BB10B08C08E199F09A00BB10B1D
:100650008050984DA449B1419093060180930501C3
:1006600020912301309124014091250150912601D0
:100670008091840090918500A0E0B0E0820F931FEC
:10068000A41FB51F80931F0190932001A093210107
:10069000B093220120918400309185008091110156
:1006A000909112018217930708F4409880911301EA
:1006B000909114018217930708F4419880911501D5
:1006C000909116018217930708F44298E09328014D
:1006D000EF91BF91AF919F918F917F916F915F91BA
:1006E0004F913F912F911F910F91FF90EF900F909D
:1006F0000FBE0F901F9018951F920F920FB60F927A
:1007000011242F933F934F935F936F937F938F9316
:100710009F93AF93BF93EF93FF938091B900887F2E
:10072000803909F44CC08139A0F4803709F43FC006
:10073000813730F48036D9F1883609F0B8C037C037
:100740008038E9F1883809F457C0883709F0AFC01C
:100750002EC0803B99F0813B48F4803A09F4A3C055
:10076000883A61F0883909F0A2C046C0803CC9F0DF
:10077000883CB9F0883B09F09AC002C010923F0152
:1007800090913F01E92FF0E0E95FFE4F8081809377
:10079000BB009F5F90933F0180913F01893041F5FD
:1007A0001EC08091BC008F7C8093BC0021C08091D2
:1007B000BC00806C8093BC0010923F017DC0809192
:1007C0003F01E82FF0E09091BB00EB5CFE4F90837F
:1007D0008F5F80933F0180913F01873049F4809182
:1007E000BC008F7B8093BC008091BC00806862C09D
:1007F0008091BC00806C5EC0E0913F01F0E0809190
:10080000BB00EB5CFE4F80838091BC00806C8093CA
:10081000BC0080913501833409F04EC090913C01B9
:1008200090958BB18F718BB98BB19295990F907E0A
:10083000982B9BB980913C0186958695869520DC06
:10084000809136019091370124E130E0AC01429F64
:10085000C001439F900D529F900D1124909312015F
:10086000809311018091380190913901AC01429F30
:10087000C001439F900D529F900D1124909314013D
:100880008093130180913A0190913B01AC01429F0A
:10089000C001439F900D529F900D1124909316011B
:1008A0008093150109C08091BC00846803C0109238
:1008B000BC0085EC8093BC00FF91EF91BF91AF919C
:1008C0009F918F917F916F915F914F913F912F9168
:0E08D0000F900FBE0F901F901895F894FFCF59
:00000001FF
